:100000000C942B050C9472050C9460060C947205EC
:100010000C9472050C9472050C9472050C94720584
:100020000C9472050C9472050C945F0D0C94310EB7
:100030000C941C1D0C9472050C9472050C947205A2
:100040000C9472050C9472050C9472050C94720554
:100050000C9472050C94901D0C9472050C9472050E
:100060000C9472050C9472050C9472050C94720534
:100070000C9472050C9472050C9472050C94720524
:100080000C9472050C9472050C9472050C94720514
:100090000C9472050C9472050C9472050C94720504
:1000A0000C9472050C9472050C9472059E0EC00E91
:1000B000AE0FC00EAE0F050F280FAE0F7D0F900FC5
:1000C000E512E512141314137213B013CA15CA15EE
:1000D000C913CA15CA14CA149E15CA15CA15B5156E
:1000E00000291E1F20212223242526272D2E2A2BDE
:1000F000141A0815171C180C12132F3028E00416B8
:1001000007090A0B0D0E0F333435E1311D1B06199B
:10011000051110363738E500E22C393A3B3C3D3EBC
:100120003F4041424353475F6061565C5D5E5759B3
:100130005A5B6263460000000000000000000000FF
:1001400000000000000000000000000000000000AF
:10015000000000000000000000000000000000009F
:1001600046756C6C002530325820004B6579626F03
:100170006172642073746172742E0A004B65796237
:100180006F61726420696E69742E0A005B445D00C1
:100190005B435D002C035800540020006B00650099
:1001A000790062006F00610072006400200063004B
:1001B0006F006E00760065007200740065007200CA
:1001C00000000E0374002E006D002E006B002E0048
:1001D00000000403090409028D00050100A0320992
:1001E0000400000103010100092111010001224066
:1001F000000705810308000A090401000103010248
:1002000000092111010001224D00070582030800A9
:100210000A09040200010300000009211101000184
:100220002236000705830308000A090403000203BD
:1002300000000009211101000122220007058403AA
:100240002000010705040320000109040400010344
:100250000000000921110100012239000705850372
:100260002000011201100100000008EDFE126501DE
:10027000000102000105010906A101050719E02995
:10028000E715002501950875018102050819012966
:1002900005950575019102950175039101050719F1
:1002A0000029F71500250195F875018102C0063176
:1002B000FF0974A1010975150026FF009520750836
:1002C00081020976150026FF00952075089102C06D
:1002D00005010980A101850216810026B7001A8157
:1002E000002AB700751095018100C0050C0901A115
:1002F000018503160100269C021A01002A9C027542
:100300001095018100C005010902A1010901A100A8
:1003100005091901290515002501950575018102B9
:100320009501750381010501093009311581257F8A
:1003300095027508810609381581257F9501750894
:100340008106050C0A38021581257F950175088103
:1003500006C0C005010906A101050719E029E71536
:100360000025019508750181029501750881010537
:1003700008190129059505750191029501750391EB
:10038000010507190029FF150026FF0095067508CD
:100390008100C0636F6E73756D65723A20253034CD
:1003A000580A0073797374656D3A20253034580A01
:1003B000000A002530325820006B6579626F617247
:1003C000643A20004C45443A20253032580A002532
:1003D0003032583A202530386225730A00722F6374
:1003E0002030313233343536370A0064656C5F6B48
:1003F00065795F6269743A2063616E277420646571
:100400006C3A20253032580A006164645F6B65796C
:100410005F6269743A2063616E2774206164643A94
:1004200020253032580A00290A002575002F0025A2
:1004300075005D280025640020002564002000254B
:10044000640020002564007C0025303258006D6F68
:100450007573656B6579205B62746E7C782079209A
:100460007620685D287265702F61636C293A205B85
:10047000006D6B5F776865656C5F74696D655F744F
:100480006F5F6D6178203D2025640A006D6B5F779A
:100490006865656C5F6D61785F7370656564203D4C
:1004A0002025640A006D6B5F74696D655F746F5F12
:1004B0006D6178203D2025640A006D6B5F6D617869
:1004C0005F7370656564203D2025640A006D6B5F75
:1004D000696E74657276616C203D2025640A006D3A
:1004E0006B5F64656C6179203D2025640A006D6B4B
:1004F0005F776865656C5F74696D655F746F5F6D6C
:100500006178203D2025640A006D6B5F7768656522
:100510006C5F6D61785F7370656564203D20256454
:100520000A006D6B5F74696D655F746F5F6D6178F4
:10053000203D2025640A006D6B5F6D61785F7370EC
:10054000656564203D2025640A006D6B5F696E74EB
:10055000657276616C203D2025640A006D6B5F64D6
:10056000656C6179203D2025640A000A002575002C
:10057000363A20776865656C5F74696D655F746F86
:100580005F6D61783A20000A00257500353A2077C2
:100590006865656C5F6D61785F73706565643A204E
:1005A000000A00257500343A2074696D655F746F28
:1005B0005F6D61783A20000A00257500333A206D9E
:1005C00061785F73706565643A20000A00257500E4
:1005D000323A20696E74657276616C286D73293ABF
:1005E00020000A00257500313A2064656C61792885
:1005F0002A31306D73293A20000A092D2056616C8A
:10060000756573202D0A004D3E004D25643E200087
:100610003F007365742064656661756C740A0043FD
:100620003E200077686572652064656C74613A20CD
:10063000637572736F723D25642C20776865656CF5
:100640003D25640A53656520687474703A2F2F65E0
:100650006E2E77696B6970656469612E6F72672FA2
:1006600077696B692F4D6F7573655F6B6579730A79
:10067000000A092D204D6F7573656B6579202D0A71
:100680004553432F713A09717569740A313A096407
:10069000656C6179282A31306D73290A323A09690B
:1006A0006E74657276616C286D73290A333A096D30
:1006B00061785F73706565640A343A0974696D65C1
:1006C0005F746F5F6D61780A353A09776865656CAC
:1006D0005F6D61785F73706565640A363A097768A3
:1006E00065656C5F74696D655F746F5F6D61780AD5
:1006F0000A703A097072696E742076616C75657360
:100700000A643A097365742064656661756C747374
:100710000A75703A092B310A646F776E3A092D31E8
:100720000A706775703A092B31300A7067646F7709
:100730006E3A092D31300A0A7370656564203D20D8
:1007400064656C7461202A206D61785F73706565E3
:1007500064202A2028726570656174202F207469D6
:100760006D655F746F5F6D6178290A003F004D3ED3
:100770002000433E20004C25640A000A092D204336
:100780006F6E736F6C65202D0A4553432F713A09C4
:10079000717569740A6D3A096D6F7573656B65796A
:1007A0000A000A092D204D61676963202D0A643A09
:1007B0000964656275670A783A096465627567203D
:1007C0006D61747269780A6B3A09646562756720B5
:1007D0006B6579626F6172640A6D3A09646562756E
:1007E00067206D6F7573650A763A0976657273696D
:1007F0006F6E0A733A097374617475730A633A0908
:10080000636F6E736F6C65206D6F64650A302D3495
:100810003A096C61796572302D34284631302D46A5
:1008200034290A506175733A09626F6F746C6F6195
:100830006465720A6E3A094E4B524F0A003F004EF1
:100840004B524F3A206F66660A004E4B524F3A2089
:100850006F6E0A0074696D65725F72656164333230
:1008600028293A202530346C580A006B6579626F6C
:100870006172645F6E6B726F3A2025580A006B6577
:1008800079626F6172645F69646C653A2025580A09
:10089000006B6579626F6172645F70726F746F6311
:1008A0006F6C3A2025580A00686F73745F6B657926
:1008B000626F6172645F6C65647328293A20255801
:1008C0000A000A092D20537461747573202D0A00E3
:1008D0004743433A20342E392E32204156522D4C74
:1008E0004942433A20312E382E3073766E204156DD
:1008F000525F415243483A20617672350A004F50A8
:1009000054494F4E533A204C554641204D4F555374
:10091000454B45592045585452414B455920434F6A
:100920004E534F4C4520434F4D4D414E44204E4B6E
:10093000524F20343039360A004255494C443A204F
:1009400065336437623530202831333A35343A31F3
:1009500037205365702032332032303138290A0075
:100960005649443A2030784645454428742E6D2E29
:100970006B2E29205049443A2030783635313228C0
:100980005854206B6579626F61726420636F6E7674
:10099000657274657229205645523A20307830309D
:1009A00030310A00444553433A20636F6E766572D6
:1009B00074205854206B6579626F61726420746F83
:1009C000205553420A000A092D2056657273696F3B
:1009D0006E202D0A000A6D6F7573653A206F66668A
:1009E0000A000A6D6F7573653A206F6E0A000A6B14
:1009F0006579626F6172643A206F66660A000A6BFD
:100A00006579626F6172643A206F6E0A000A6D61E7
:100A1000747269783A206F66660A000A6D617472B2
:100A200069783A206F6E0A000A64656275673A2039
:100A30006F6E0A000A64656275673A206F66660A1F
:100A4000000A0A626F6F746C6F616465722E2E2EDD
:100A50002000433E200011241FBECFEFDAE0DEBFAE
:100A6000CDBF04B603FE27C08091EC039091ED0347
:100A7000A091EE03B091EF038730904BA740B04BAD
:100A8000D1F41092EC031092ED031092EE03109249
:100A9000EF0314BE84B7877F84BF0FB6F894A89580
:100AA00080916000886180936000109260000FBEAA
:100AB000E0E0F8E3099511E0A0E0B1E0E2E5FDE453
:100AC00002C005900D92AA38B107D9F723E0AAE831
:100AD000B1E001C01D92AC3EB207E1F70E94120ADC
:100AE0000C94A7260C940000FF93EF93E0918A01E9
:100AF000F0918B01309709F00995EF91FF910895DE
:100B0000FC018591803011F0EFDFFBCF0895FF27C6
:100B1000E0E230E247FF0CC0419597FF09C0EDE2EB
:100B20006095709580959095611D711D811D911D39
:100B300027FF02C0219530E350E2AA27660F771FF6
:100B4000881F991FAA1FA41710F0A41B63955A951C
:100B5000A9F7AA3008F0A95FA05DAF93F3956115DE
:100B600071058105910541F7ED3211F4EF93F3958D
:100B7000F21718F43F93F395FBCF8F91B5DFFA95F9
:100B8000E1F70895E991F9918591803021F085325E
:100B900019F0AADFF9CF089520E0E8945591553275
:100BA000C1F3503311F4689455915A3348F45053BB
:100BB00090F3220F022E220F220F200D250FF4CFCB
:100BC0000EF4219589919991533619F3533729F1F0
:100BD000533559F1BC0188279927E8945C3621F4F4
:100BE0008991999168945591543639F446EF7EF085
:100BF00077FF0DC08FEF9FEF0AC055374AE039F0FD
:100C0000583540E121F0523642E009F00895FF9353
:100C1000EF937DDFEF91FF91B7CFFF93EF93FC014F
:100C200081918030B9F360DFFBCFFF93EF9368DFF2
:100C3000F1CFDF93CF93CDB7DEB72596A3DFCF916A
:100C4000DF910895E9E6F0E0808188608083E9988B
:100C50002F98279A2FEF89E698E121508040904005
:100C6000E1F700C0000027985898509A5998519A77
:100C70002FEF89EF90E0215080409040E1F700C0D5
:100C800000005198599A5098589AE19AE99A089513
:100C90009091030180910201891781F0E091000198
:100CA000F0910101E90FF11D80819F5F2091040106
:100CB0009223909303015098589A089580E00895E4
:100CC0001F920F920FB60F9211242F933F934F93C1
:100CD0005F936F937F938F939F93AF93BF93EF93A4
:100CE000FF9329B1217090918D01992319F09930CA
:100CF00058F403C0211108C04AC080918C01869528
:100D00002111806880938C0181E0890F80938D018F
:100D10009830E9F560918C018091020190E0AC017E
:100D20004F5F5F4F30910401232F30E024233523A0
:100D30004091030150E02417350781F02091000114
:100D400030910101F901E80FF91F608380910201E0
:100D50008F5F9091040189238093020180910201A9
:100D600090E001962091040130E0822393232091AA
:100D7000030130E08217930731F45898509A80E6C7
:100D800091E00E94800510928D0110928C01FF91DC
:100D9000EF91BF91AF919F918F917F916F915F91F3
:100DA0004F913F912F910F900FBE0F901F9018956C
:100DB000CF93DF93D82FD770C82FC695C695C69509
:100DC0006D2F8C2F0E94331181110DC0EC2FF0E09C
:100DD000E156FE4F81E090E001C0880FDA95EAF716
:100DE0009081892B8083DF91CF910895CF93DF93FA
:100DF000D82FD770C82FC695C695C6956D2F8C2F46
:100E00000E943311882371F0EC2FF0E0E156FE4F81
:100E100081E090E001C0880FDA95EAF78095908133
:100E200089238083DF91CF9108958091CE038160E3
:100E30008093CE030E942206EFE9F1E080E18E0F5D
:100E400011928E13FDCF0895CF93DF931F92CDB7EC
:100E5000DEB70E944806882309F473C09091CE0340
:100E600090FF0EC01F928F9325E631E03F932F93A2
:100E700089830E9419060F900F900F900F9089811F
:100E800090919E01923009F442C028F4992351F0C8
:100E90009130B1F052C0933009F443C0943009F45A
:100EA00046C04BC0803E21F0813E31F482E036C026
:100EB00081E080939E0146C087FF36C08F773AC09D
:100EC0008633D9F118F48A3229F437C08A3AA9F165
:100ED000863B99F187FD0DC08C51883430F4E82FA2
:100EE000F0E0E25EFE4F808101C080E00E94D80603
:100EF00024C0E82FEF77EC51E83428F4F0E0E25E0C
:100F0000FE4F808101C080E00E94F60616C08D3140
:100F100021F08D3991F484E001C083E080939E013B
:100F20000EC0853451F485E50E94D80608C085348A
:100F300021F485E50E94F60602C010929E0181E030
:100F400001C080E00F90DF91CF910895E82FF0E08D
:100F5000E156FE4F80810895EFE9F1E080E18E0FC8
:100F600011928E13FDCF089508958091D2020895B5
:100F7000CF93DF9300D01F92CDB7DEB79C01809155
:100F8000E303843019F593E099833B832A8390939C
:100F9000E9008FEF9091E800815095FD06C095ED36
:100FA0009A95F1F700008111F5CF8091E80085FF57
:100FB0000DC040E050E063E070E0CE0101960E9479
:100FC0004F0B8091E8008E778093E8000F900F9090
:100FD0000F90DF91CF910895CF93DF9300D01F92B0
:100FE000CDB7DEB72091E303243021F522E0298339
:100FF0009B838A8383E08093E9008FEF9091E800E0
:10100000815095FD06C095ED9A95F1F7000081118C
:10101000F5CF8091E80085FF0DC040E050E063E02F
:1010200070E0CE0101960E944F0B8091E8008E7710
:101030008093E8000F900F900F90DF91CF9108956B
:101040002091E3032430F1F422E02093E9002FEF14
:101050003091E800215035FD06C035ED3A95F1F7A5
:1010600000002111F5CF2091E80025FF0BC040E0E2
:1010700050E065E070E00E944F0B8091E8008E77B1
:101080008093E8000895CF93DF932091E303243009
:1010900009F04AC0EC01809114018823E1F08091AD
:1010A00015018823C1F085E08093E90081E8815033
:1010B00049F09091E80095FD05C09AE29A95F1F704
:1010C00000C0F5CF8091E80085FF2EC040E050E0E1
:1010D00060E270E019C081E08093E90081E881500E
:1010E00059F09091E80095FD07C0EFE3F1E03197EA
:1010F000F1F700C00000F3CF8091E80085FF14C035
:1011000040E050E068E070E0CE010E944F0B80911B
:10111000E8008E778093E80080E2FE01A2EBB2E067
:1011200001900D928A95E1F7DF91CF9108950FB666
:1011300007FE45C09091E303943009F040C09091C0
:10114000E9009F703091EC00232F217030FD20E8E2
:10115000922B24E02093E9002091EB0020FF2CC08B
:101160002091EE0027FF28C020910801309107014F
:10117000321709F449C03091E80035FF1DC0E091F5
:101180000501F0910601E20FF11D40812F5F3091C2
:1011900009012323209308014093F1002091E800E6
:1011A00025FDE2CF2091E80020FFDECF2091E8006E
:1011B0002E772093E800D8CF9F709093E90020917C
:1011C000070130E0B9016F5F7F4F90910901492F0E
:1011D00050E0462357236091080170E046175707F7
:1011E00089F04091050150910601FA01E20FF31FC9
:1011F0008083809107018F5F9091090189238093FB
:1012000007010BC08FEF08952091E80025FFD4CF90
:101210008093F1009F709093E90080E0089580E949
:1012200091E00E9480058091E203811109C00E9433
:10123000E40C0E94410D8091E20084608093E20002
:1012400008958CE891E00E9480051092E2030895D1
:101250000895089542E061EC81E00E945E0C42E056
:1012600061EC82E00E945E0C42E061EC83E00E944F
:101270005E0C42E261EC84E00E945E0C42E261ECB2
:1012800085E00C945E0C8091E503833009F455C031
:1012900030F4813071F0823009F48EC008958A30C4
:1012A00009F47AC08B3009F460C0893009F09CC021
:1012B00020C08091E403813A09F096C08091E80053
:1012C000877F8093E8008091E8039091E903892B60
:1012D00021F460E282EB92E003C060E080E090E005
:1012E00070E00E949A0B8091E8008B778093E80071
:1012F00008958091E403813209F076C08091E8037B
:101300009091E903009719F0049709F06DC080915E
:10131000E800877F8093E8008091E80082FD05C0A7
:101320008091E3038111F8CF5FC08091F100809339
:10133000D2028091E8008B7753C08091E403813A18
:1013400009F052C08091E8039091E903892B09F0DC
:101350004BC08091E800877F8093E8008091E8008F
:1013600080FFFCCF8091140136C08091E40381326C
:10137000D9F58091E8039091E903892BA9F5809133
:10138000E800877F8093E8000E94930C8091E60339
:10139000809314010C94EC158091E403813221F5C3
:1013A0008091E800877F8093E8000E94930C8091F1
:1013B000E7038093D30208958091E403813AA1F476
:1013C0008091E800877F8093E8008091E80080FFAB
:1013D000FCCF8091D3028093F1008091E8008E775A
:1013E0008093E8000C94930C0895089508958091DB
:1013F000D2028093B1011092D20280E00E94B40721
:101400000E94AC070C94EC150C94F7090E94DB1CAD
:101410008091E103882329F00E94041D81110C941E
:10142000390B0895CF9384B7877F84BF0FB6F894A4
:10143000A8958091600088618093600010926000A0
:101440000FBE90E080E80FB6F8948093610090930F
:1014500061000FBE87E998E00E94AC1C8AE091E031
:101460000E94C60F8CE791E00E9480050E94F5095A
:101470000E9487100E94E40C0E94410D8091E200BE
:1014800084608093E20078948091E3038430E1F7F4
:101490000E9489108091CE0380FD08C00E94F60949
:1014A0008BE691E00E948005C4E018C081ED97E0D2
:1014B0000197A1F3EFE9FFE03197F1F700C00000D9
:1014C000F7CF0E948D108091E4009091E50020916B
:1014D000AF013091B0012817390739F48091E30347
:1014E000853079F70E94060AF9CF8091E400909147
:1014F000E5009093B0018093AF018091E3038430C5
:1015000069F78091E9008F702091EC00922F917023
:1015100020FD90E8892BC093E9009091EB0090FFAB
:1015200043C09091EE0097FF3FC090910801209139
:101530000701291709F12091E80025FF1DC0E0915E
:101540000501F0910601E90FF11D30819F5F2091A7
:1015500009019223909308013093F1009091E800E3
:1015600095FDE3CF9091E80090FFDFCF9091E800E8
:101570009E779093E800D9CF9091F3002091F200EC
:1015800030E0392B232B81F09091E80090FF0CC0C4
:101590009091E80095FF03C01092F100F9CF90916F
:1015A000E8009E779093E8008F708093E90096CFD3
:1015B0000E94181D8091B1018093D20208950C946D
:1015C000D80A292F332723303105C9F064F421309C
:1015D000310581F02230310509F043C08DE890E0FB
:1015E00026ED31E042C021323105F1F022323105E1
:1015F00041F137C082E190E023E632E036C099271E
:101600008130910541F08230910541F0892B49F5F7
:10161000E2EDF1E005C0E2ECF1E002C0E4E9F1E066
:10162000849190E09F0121C06530D8F4E62FF0E06E
:10163000EE0FFF1FEB58FE4F2081318189E090E0D3
:1016400014C0653070F470E0FB01EE0FFF1FE55928
:10165000FE4F20813181FB01EA59FE4F808190E0ED
:1016600004C080E090E020E030E0FA013183208384
:10167000089580E189BD82E189BD09B400FEFDCFF6
:101680008091D8008F7D8093D8008091E0008260A7
:101690008093E0008091E00081FDFCCF0895CF921F
:1016A000DF92EF92FF920F931F93CF93DF93EC01A2
:1016B0008B016A010E94B20C811133C0C114D104A4
:1016C00039F0F60180819181081B190BC80FD91FD1
:1016D000E12CF12C0115110519F18091E80085FD2F
:1016E00016C08091E8008E778093E800C114D10481
:1016F00049F0F60180819181E80EF91EF182E082C5
:1017000085E00FC00E94B20C882321F30AC08991A2
:101710008093F10001501109FFEFEF1AFF0ADACFB1
:1017200080E0DF91CF911F910F91FF90EF90DF90BC
:10173000CF9008952091EA033091EB0326173707E5
:1017400048F06115710539F42091E8002E77209357
:10175000E80001C0B90140E061157105A9F12091CF
:10176000E303222309F443C0253009F442C0209149
:10177000E80023FD40C02091E80022FD32C0209106
:10178000E80020FFE9CF4091F3002091F20030E023
:10179000342BFC01CF016115710559F0283031055A
:1017A00040F481918093F100615071092F5F3F4FA8
:1017B000F1CF41E02830310509F040E02091E80008
:1017C0002E772093E800C8CF4111C9CF0AC080917D
:1017D000E303882361F0853061F08091E80083FDA8
:1017E0000AC08091E80082FFF2CF80E0089582E095
:1017F000089583E0089581E008952091EA033091EF
:10180000EB032617370748F06115710539F420916D
:10181000E8002E772093E80001C0B901FC0120E028
:101820006115710591F18091E303882309F440C0AB
:10183000853009F43FC08091E80083FD3DC0809170
:10184000E80082FD2FC08091E80080FFE9CF209161
:10185000F3008091F20090E0922B6115710559F030
:101860008830910540F424912093F1003196615025
:1018700071090196F2CF21E0089709F020E08091EC
:10188000E8008E778093E800CBCF2111CCCF0AC03F
:101890008091E303882361F0853061F08091E80056
:1018A00083FD0AC08091E80082FFF2CF80E00895B6
:1018B00082E0089583E0089581E00895982F97309D
:1018C00058F59093E900981739F07091EC00209149
:1018D000ED005091F00003C0242F762F50E021FF3F
:1018E00019C03091EB003E7F3093EB003091ED005A
:1018F0003D7F3093ED003091EB0031603093EB0091
:101900007093EC002093ED005093F0002091EE00D6
:1019100027FF07C09F5FD3CF8F708093E90081E0DE
:10192000089580E008958091E40387FF11C08091BD
:10193000E80082FD05C08091E3038111F8CF11C05A
:101940008091E8008B770BC08091E303882349F0F6
:101950008091E80080FFF8CF8091E8008E77809337
:10196000E80008952091E4003091E50095E640916B
:10197000EC00842F817040FF22C08091E80080FD40
:101980001CC08091E303882391F0853091F0809111
:10199000EB0085FD10C04091E4005091E500421736
:1019A000530729F39A01915011F784E0089582E0DA
:1019B000089583E0089581E0089580E008954091BE
:1019C000E80042FFDECF08950E94520D0E945A0D9A
:1019D000E0EEF0E0808181608083E8EDF0E08081DE
:1019E0008F77808319BCA7EDB0E08C918E7F8C93AC
:1019F00080818F7E80831092E20308950F931F935E
:101A0000CF93DF930E94520D0E945A0DC8EDD0E093
:101A100088818F77888388818068888388818F7D9B
:101A2000888319BC1092E3031092DF031092E10344
:101A30001092E00300EE10E0F80180818B7F80833C
:101A400088818160888342E060E080E00E945E0CD3
:101A5000E1EEF0E080818E7F8083E2EEF0E0808135
:101A600081608083808188608083F80180818E7F9F
:101A70008083888180618883DF91CF911F910F914E
:101A80000895E8EDF0E080818F7E8083E7EDF0E05F
:101A900080818160808384E082BF81E08093E20363
:101AA0000C94FE0CE8EDF0E080818E7F8083109234
:101AB000E20008951092DA001092E10008951F925A
:101AC0000F920FB60F9211242F933F934F935F9372
:101AD0006F937F938F939F93AF93BF93EF93FF93F6
:101AE0008091E10082FF0BC08091E20082FF07C07D
:101AF0008091E1008B7F8093E1000E942909809111
:101B0000DA0080FF1FC08091D80080FF1BC0809149
:101B1000DA008E7F8093DA008091D90080FF0DC0BB
:101B200080E189BD82E189BD09B400FEFDCF81E07D
:101B30008093E3030E940F0905C019BC1092E303D0
:101B40000E9421098091E10080FF19C08091E2008C
:101B500080FF15C08091E2008E7F8093E20080912B
:101B6000E20080618093E2008091D80080628093DF
:101B7000D80019BC85E08093E3030E94040A809199
:101B8000E10084FF30C08091E20084FF2CC080E13E
:101B900089BD82E189BD09B400FEFDCF8091D800E6
:101BA0008F7D8093D8008091E1008F7E8093E1004B
:101BB0008091E2008F7E8093E2008091E20081605C
:101BC0008093E2008091DF03882311F084E007C056
:101BD0008091E30087FD02C081E001C083E0809333
:101BE000E3030E94DF0A8091E10083FF29C0809116
:101BF000E20083FF25C08091E100877F8093E100B0
:101C000082E08093E3031092DF038091E1008E7FF6
:101C10008093E1008091E2008E7F8093E2008091CA
:101C2000E20080618093E20042E060E080E00E9498
:101C30005E0C8091F00088608093F0000E9428097B
:101C4000FF91EF91BF91AF919F918F917F916F9194
:101C50005F914F913F912F910F900FBE0F901F906A
:101C600018951F920F920FB60F9211242F933F9346
:101C70004F935F936F937F938F939F93AF93BF9394
:101C8000CF93DF93EF93FF93C091E900CF708091E2
:101C9000EC00D82FD17080FDD0E81092E90080913F
:101CA000F000877F8093F00078940E94750E109268
:101CB000E9008091F00088608093F000CD2BCF7018
:101CC000C093E900FF91EF91DF91CF91BF91AF9168
:101CD0009F918F917F916F915F914F913F912F9144
:101CE0000F900FBE0F901F9018951F93CF93DF9307
:101CF000CDB7DEB7AA970FB6F894DEBF0FBECDBF43
:101D0000E4EEF3E088E08E0F9091F10091938E1352
:101D1000FBCF0E9443098091E80083FF1FC180919F
:101D2000E4039091E503492F50E04A30510508F053
:101D300015C1FA01EA5AFF4F0C948D26803881F0C4
:101D4000823809F00BC18091E8038F708093E9001D
:101D50008091EB0085FB882780F91092E90006C08E
:101D60008091E0039091E103911182609091E800ED
:101D7000977F9093E8008093F1001092F100C8C023
:101D8000282F2D7F09F0EAC0882319F0823061F0F6
:101D9000E5C08091E603813009F0E0C0933009F09E
:101DA00080E08093E1032BC08091E603811127C07E
:101DB0008091E8038F7009F4D1C08093E9002091ED
:101DC000EB0020FF1CC0933021F48091EB00806277
:101DD00014C09091EB0090619093EB0021E030E013
:101DE000A90102C0440F551F8A95E2F74093EA000B
:101DF0001092EA008091EB0088608093EB001092D3
:101E0000E9008091E800877F86C08111A7C010910A
:101E1000E6031F778091E3008078812B8093E300B5
:101E20008091E800877F8093E8000E94930C809166
:101E3000E80080FFFCCF8091E30080688093E3009E
:101E4000111102C082E001C083E08093E30386C0E9
:101E50008058823008F082C08091E6039091E703B9
:101E60008C3D53E0950779F583E08A838AE2898384
:101E70004FB7F894DE01139620E03EE051E2E32FE5
:101E8000F0E050935700E49120FF03C0E295EF701B
:101E90003F5FEF708E2F90E0EA3010F0C79601C0E0
:101EA000C0968D939D932F5F243149F74FBF80914A
:101EB000E800877F8093E8006AE270E0CE01019637
:101EC0000E949A0B14C0AE014F5F5F4F6091E80310
:101ED0000E94E10ABC01892B09F440C09091E800FE
:101EE000977F9093E80089819A810E94FD0B8091F1
:101EF000E8008B778093E80031C0803879F58091D5
:101F0000E800877F8093E8008091DF038093F100F1
:101F10008091E8008E778093E8000E94930C1EC0A9
:101F200081111CC09091E6039230C0F48091E800CA
:101F3000877F8093E8009093DF030E94930C809149
:101F4000DF03811106C08091E30087FD02C081E0BC
:101F500001C084E08093E3030E942A098091E80095
:101F600083FF0AC08091E800877F8093E80080911A
:101F7000EB0080628093EB00AA960FB6F894DEBF68
:101F80000FBECDBFDF91CF911F9108959093D902DD
:101F90008093D8020895E091D802F091D902309749
:101FA00021F00190F081E02D099480E00895EF92F6
:101FB000FF920F931F93CF93DF93E091D802F0919C
:101FC000D9023097B1F18C010280F381E02D09959F
:101FD0008091CE0382FF2DC080FF04C089EB93E087
:101FE0000E948005E80110E283EBE82E83E0F82EE2
:101FF0008091CE0380FF0BC088811F928F93FF9248
:10200000EF920E9419060F900F900F900F901150B1
:1020100021961111EDCF8091CE0380FF0AC081EB94
:1020200093E0DF91CF911F910F91FF90EF900C946F
:102030008005DF91CF911F910F91FF90EF90089550
:10204000E091D802F091D902309721F00480F58117
:10205000E02D09940895CF93DF93EC018091D6028F
:102060009091D702C817D90709F1D093D702C0932E
:10207000D602E091D802F091D9023097B9F00680EB
:10208000F781E02DCE0109958091CE0382FF0EC02D
:1020900080FF0CC0DF93CF9383EA93E09F938F93ED
:1020A0000E9419060F900F900F900F90DF91CF9123
:1020B0000895CF93DF93EC018091D4029091D502E3
:1020C000C817D90709F1D093D502C093D402E09183
:1020D000D802F091D9023097B9F00084F185E02D53
:1020E000CE0109958091CE0382FF0EC080FF0CC007
:1020F000DF93CF9383E993E09F938F930E94190618
:102100000F900F900F900F90DF91CF9108950C9446
:1021100032110E94451D0C941507BF92CF92DF9299
:10212000EF92FF920F931F93CF93DF9300D000D0D5
:102130001F92CDB7DEB70E9424070BED12E0F12C01
:102140008F2D0E94A607B82EF801C080C82639F44A
:10215000F3940F5F1F4FF0E1FF12F2CF30C0809178
:10216000CE0381FD0E944E11D12CEE24E3948E2DDE
:102170008C21F9F0D982FA8281E09E2D9B2109F40D
:1021800080E08B830E944E1D8160782F9D838C831D
:1021900049815A816B818D810E94841149815A81C4
:1021A0006B817C818D810E94C81CF80190819E25E5
:1021B0009083D394EE0CF8E0DF12D9CFC9CF8FEF24
:1021C00089838A831B820E944E1D8160782F9D83A4
:1021D0008C8349815A816B818D810E9484110E9478
:1021E000C71C0E94A7201091DA020E94CB0F18177B
:1021F00041F10E94CB0F8093DA029091CE0392FFBF
:102200000EC090FF0CC01F928F9384EC93E09F93BD
:102210008F930E9419060F900F900F900F9080914E
:10222000DA020F900F900F900F900F90DF91CF91E7
:102230001F910F91FF90EF90DF90CF90BF900C9483
:10224000D91C0F900F900F900F900F90DF91CF91AE
:102250001F910F91FF90EF90DF90CF90BF90089566
:102260000C94B4070895CF93DF931F92CDB7DEB7D8
:1022700069830E94A60790E021E030E0698102C0F6
:10228000220F331F6A95E2F72823392381E0232B9D
:1022900009F480E00F90DF91CF910895EF92FF92C3
:1022A0000F931F93CF93DF938DED93E00E948005F2
:1022B000C0E0D0E08FE7E82E81E0F82E0FEC13E0CD
:1022C0008C2F0E94A6070E94B11CFF92EF921F92D2
:1022D0008F93DF93CF931F930F930E94190621963C
:1022E0008DB79EB708960FB6F8949EBF0FBE8DBFF0
:1022F000C031D10529F7DF91CF911F910F91FF9048
:10230000EF90089508950895CF93DF93CDB7DEB78A
:102310002B970FB6F894DEBF0FBECDBF942F4F831F
:10232000252F588769877A878B874A855B85452B58
:1023300021F02F3F09F59F3FF9F4DE01119686E069
:10234000FD0111928A95E9F785E0FE01379601902B
:102350000D928A95E1F749815A816B817C818D814B
:102360009E810E94C9182B960FB6F894DEBF0FBE4F
:10237000CDBFDF91CF9108954F81588569857A85CA
:102380008B850E94C81CD9CFCF93882309F4A4C0A1
:10239000C82F8CEF8C0F813A48F48C2F0E94F123C8
:1023A00081119AC08C2F0E94A11B0CC080E28C0F5F
:1023B000883058F4C77081E001C0880FCA95EAF7E9
:1023C0000E944C1CCF910C94861C8BE58C0F8330A3
:1023D00078F4C53A29F0C63A31F083E890E005C0B8
:1023E00081E890E002C082E890E0CF910C942B103D
:1023F00088E58C0F853108F06FC0C83A61F1C93AA1
:1024000069F1CA3A71F1CB3A79F1CC3A81F1CD3A1E
:1024100089F1CE3A91F1CF3A99F1C13BA1F1C03B9C
:10242000A9F1C23BB1F1C33BB9F1C43BC1F1C53B1A
:10243000C9F1C63BD1F1C73BD9F1C83BE1F1C93B7A
:10244000E9F1CA3BF1F1CB3BF9F1CC3B09F43FC0D8
:1024500080E090E03EC082EE90E03BC089EE90E0EC
:1024600038C08AEE90E035C085EB90E032C086EB54
:1024700090E02FC083EB90E02CC084EB90E029C06B
:1024800087EB90E026C08CEC90E023C08DEC90E0D0
:1024900020C083E891E01DC08AE891E01AC082E97B
:1024A00091E017C084E991E014C081E292E011C08C
:1024B00083E292E00EC084E292E00BC085E292E0FB
:1024C00008C086E292E005C087E292E002C08AE29C
:1024D00092E0CF910C945910CF910895882329F15F
:1024E0009CEF980F913A18F40E94F41B0DC090E2F3
:1024F000980F983058F4877091E001C0990F8A9531
:10250000EAF7892F0E94521C0C94861C9BE5980FB9
:10251000933020F480E090E00C942B10885A8531A1
:1025200020F480E090E00C9459100895882321F065
:102530000E944C1C0C94861C0895882321F00E9454
:10254000521C0C94861C0895BF92CF92DF92EF929A
:10255000FF920F931F93CF93DF9300D000D000D052
:10256000CDB7DEB725E0FC01DE01119601900D929A
:102570002A95E1F7FC0140815181028163817481D8
:10258000258122952F706115710509F403C35F3F02
:1025900019F44F3F09F4FEC26C01862F7D836C83D2
:1025A000602F782F8D812E830E94251B182FB92E26
:1025B0000E94241B0E94141AEB2DE295EF70F0E0AC
:1025C000E05AFF4F2E810C948D268B2D807F9B2D02
:1025D0009F70F92E882319F0F29490EFF9220023CE
:1025E00049F0FF2009F483C28F2D0E945F1C0E94D6
:1025F000861C7DC2812F0E946E12FF2009F4CAC280
:102600008F2D0E94651C26960FB6F894DEBF0FBE74
:10261000CDBFDF91CF911F910F91FF90EF90DF9091
:10262000CF90BF900C94861C8B2D807F9B2D9F702C
:10263000F92E803219F0F29480EFF822112319F06C
:10264000113009F12AC00023B1F08F2D222351F15E
:10265000213041F526960FB6F894DEBF0FBECDBFF0
:10266000DF91CF911F910F91FF90EF90DF90CF906E
:10267000BF900C946F1C222319F0213009F48AC2F8
:102680000E94721C2DC00023F1F0263008F082C297
:102690000E94491C8F2129F023C00023F9F0211149
:1026A00016C08F2D26960FB6F894DEBF0FBECDBF95
:1026B000DF91CF911F910F91FF90EF90DF90CF901E
:1026C000BF900C949612253008F064C209C0F60140
:1026D000858180FF0CC28F708583E3CF21111CC2DE
:1026E0008F2D83C12B2D26952695237030E0211543
:1026F000310521F021303105D1F04CC2002321F009
:10270000812F9B2D937002C080E090E026960FB63B
:10271000F894DEBF0FBECDBFDF91CF911F910F9117
:10272000FF90EF90DF90CF90BF900C942B10002380
:1027300021F0812F9B2D937002C080E090E02696BF
:102740000FB6F894DEBF0FBECDBFDF91CF911F91C2
:102750000F91FF90EF90DF90CF90BF900C945910A5
:10276000812F002319F00E942D1F02C00E94951F87
:1027700026960FB6F894DEBF0FBECDBFDF91CF9186
:102780001F910F91FF90EF90DF90CF90BF900C942E
:102790001A208B2D837009F07BC00111FBC1812FA2
:1027A000829586958770880F880F912F9F70C92E0C
:1027B000D12CE12CF12C082E04C0CC0CDD1CEE1C1D
:1027C000FF1C0A94D2F714FF12C04FE050E060E003
:1027D00070E004C0440F551F661F771F8A95D2F71B
:1027E000CB01BA01609570958095909503C060E02B
:1027F00070E0CB012B2D269526952370422F50E0BB
:1028000042305105D9F04330510569F16C297D29D9
:102810008E299F294130510551F126960FB6F89423
:10282000DEBF0FBECDBFDF91CF911F910F91FF9003
:10283000EF90DF90CF90BF900C94391A6C297D29CE
:102840008E299F2926960FB6F894DEBF0FBECDBF06
:10285000DF91CF911F910F91FF90EF90DF90CF907C
:10286000BF900C94531A0E94391AC701B6012696DC
:102870000FB6F894DEBF0FBECDBFDF91CF911F9191
:102880000F91FF90EF90DF90CF90BF900C941F1AA4
:10289000002319F08B2D817001C08695882309F4DF
:1028A00079C1812F829586958770880F880F912F27
:1028B0009F70C92ED12CE12CF12C082E04C0CC0C19
:1028C000DD1CEE1CFF1C0A94D2F714FF12C04FE06F
:1028D00050E060E070E004C0440F551F661F771F92
:1028E0008A95D2F7CB01BA01609570958095909545
:1028F00003C060E070E0CB012B2D26952695237058
:10290000422F50E042305105D9F04330510569F172
:102910006C297D298E299F294130510551F1269638
:102920000FB6F894DEBF0FBECDBFDF91CF911F91E0
:102930000F91FF90EF90DF90CF90BF900C94001B11
:102940006C297D298E299F2926960FB6F894DEBF23
:102950000FBECDBFDF91CF911F910F91FF90EF90F0
:10296000DF90CF90BF900C94121B0E94001BC701F8
:10297000B60126960FB6F894DEBF0FBECDBFDF912D
:10298000CF911F910F91FF90EF90DF90CF90BF906C
:102990000C94EE1A103FD1F128F480E4810F8032BC
:1029A00050F0A0C0123F09F462C008F44BC0133FBE
:1029B00009F472C097C0F12FF071FF2E8B2D8F712B
:1029C000002351F00E94871A812FFF2019F0829571
:1029D000807F68CE8F7066CE0E94A81A812FFF205C
:1029E00019F08295807F01C08F7026960FB6F894FB
:1029F000DEBF0FBECDBFDF91CF911F910F91FF9032
:102A0000EF90DF90CF90BF900C949D120023B1F017
:102A1000253008F0BFC08B2D8F7126960FB6F89425
:102A2000DEBF0FBECDBFDF91CF911F910F91FF9001
:102A3000EF90DF90CF90BF900C94CD1A263008F025
:102A4000A9C0E9CF0023A9F08B2D8F7126960FB670
:102A5000F894DEBF0FBECDBFDF91CF911F910F91D4
:102A6000FF90EF90DF90CF90BF900C94871A0023D7
:102A700059F38B2D8F7126960FB6F894DEBF0FBEDB
:102A8000CDBFDF91CF911F910F91FF90EF90DF901D
:102A9000CF90BF900C94A81A002399F08B2D8F71C2
:102AA00026960FB6F894DEBF0FBECDBFDF91CF9153
:102AB0001F910F91FF90EF90DF90CF90BF900C94FB
:102AC000721A26960FB6F894DEBF0FBECDBFDF9107
:102AD000CF911F910F91FF90EF90DF90CF90BF901B
:102AE0000C946D1A0023A9F0222309F4ADCF812F95
:102AF00026960FB6F894DEBF0FBECDBFDF91CF9103
:102B00001F910F91FF90EF90DF90CF90BF900C94AA
:102B1000C411222309F4ADCF812F26960FB6F89465
:102B2000DEBF0FBECDBFDF91CF911F910F91FF9000
:102B3000EF90DF90CF90BF900C946E124B2D4F70A2
:102B4000612FC6010E94D71D26960FB6F894DEBFEE
:102B50000FBECDBFDF91CF911F910F91FF90EF90EE
:102B6000DF90CF90BF900C946D194B2D4F70612F5B
:102B7000C60126960FB6F894DEBF0FBECDBFDF911B
:102B8000CF911F910F91FF90EF90DF90CF90BF906A
:102B90000C94DA1D26960FB6F894DEBF0FBECDBF9B
:102BA000DF91CF911F910F91FF90EF90DF90CF9029
:102BB000BF9008950E946C1C0E943B1C0E94861CC2
:102BC0000E944C210E941A2080E090E00E942B106D
:102BD00080E090E00C9459100E945C1C0C94DA1573
:102BE000CF93DF9300D000D01F92CDB7DEB7942FE4
:102BF0004983252F5A836B837C838D834C815D8130
:102C0000452B39F12F3F11F49F3F19F149815A812A
:102C10006B817C818D810E94251B292F22952F702D
:102C200030E02C30310504F52A3031055CF42250B7
:102C300031092230310568F4853A80F4843090F40B
:102C4000823080F0883E38F4803E60F48450813ACF
:102C500048F080E014C0803FE1F704C090E2980F94
:102C6000983080F781E00BC02C30310521F493FBC4
:102C7000882780F904C02F303105C9F3EACF0F90BF
:102C80000F900F900F900F90DF91CF910895CF93F9
:102C9000DF9300D000D01F92CDB7DEB70F900F901A
:102CA0000F900F900F90DF91CF910895CF93DF9306
:102CB00000D000D000D0CDB7DEB726960FB6F8947E
:102CC000DEBF0FBECDBFDF91CF9108951F93CF938D
:102CD000DF93C091EB0216E08091EC02C81799F0E7
:102CE000D0E01C9FF0011D9FF00D1124E351FD4F1A
:102CF0004081518162817381848195810E94561641
:102D00002196C770E9CFDF91CF911F91089540912F
:102D10001D0350911E0360911F0370912003809149
:102D20002103909122030C945616809122038295E0
:102D30008F7009F054C080911F03882309F44FC09D
:102D40008091EB02A091EC0260911D0370911E0333
:102D50004091200350912103B6E08A1709F43FC047
:102D600090E041155105C1F17F3F11F46F3FA1F192
:102D7000B89FF001B99FF00D1124E351FD4F21815F
:102D800072132AC02081621327C02281211124C01E
:102D9000238134812417350710F421503109241B75
:102DA000350B283C3105C0F4209122032F7020619F
:102DB0002093220326E0289FF001299FF00D112483
:102DC000EE50FD4F80818F70806180838DE193E0B4
:102DD0000E94A4120C94661601968770BECF0895C7
:102DE000BF92CF92DF92EF92FF920F931F93CF93F8
:102DF000DF93CDB7DEB761970FB6F894DEBF0FBE95
:102E0000CDBF7C0185E0F701DE011D9601900D929A
:102E10008A95E1F7D7014C9111965C911197129622
:102E2000DC90129713960D911C91149730911D030D
:102E300060911E038091200390912103009709F473
:102E400077C16F3F19F43F3F09F472C1B0901F037F
:102E5000BB2009F4C5C0209122030817190728F0E8
:102E6000F801E81BF90BCF0104C080959095800F05
:102E7000911FCC24C394883C910580F0C12C207F05
:102E800009F0CCC0702F198B088B6D2D89890E9499
:102E900047168DE193E00E94A412B6C0822F807F76
:102EA00009F047C0651314C0341312C0D11010C00C
:102EB0002F702061209322030E9487168DE193E0FA
:102EC0000E94A41280912203D70115968C932FC0E3
:102ED0000115110519F15F3F11F44F3FF9F0CD2CA9
:102EE000D1101CC08091EB022091EC0236E08217D9
:102EF00009F45CC090E0389FF001399FF00D112477
:102F0000E351FD4F6181561306C06081461303C033
:102F10006281611103C001968770E9CFCD2CDD205D
:102F200009F426C180912203816080932203C12C81
:102F30001FC1651308C0341306C0D11004C08091AE
:102F40002203D701C9C04D875E87DF86702F198B9A
:102F5000088B6D2D89890E94F0158823E9F1DD2009
:102F6000D9F120912203822F82958F7090E00297F1
:102F700074F080911D0390911E0398878F831986AA
:102F80001B870A872C87CE0107960E94A41286E031
:102F9000F701ADE1B3E001900D928A95E1F70E944F
:102FA00095160E948716CC24C394E2C0702F198B0B
:102FB000088B60E089890E94251B292F22952F709C
:102FC00030E0223031050CF0C7C09F7009F0C1C05D
:102FD000805E883008F4CCC0C7010E94A412E3CF01
:102FE0000817190708F456C0F801E81BF90BCF01C0
:102FF000883C910508F453C0C12C702F198B088BA5
:103000006D2D89890E944716EDE1F3E086E0DF012E
:103010001D928A95E9F70E948716AAC0651314C00D
:10302000341312C0D11010C080912203F7018583A0
:10303000C7010E94A41286E0EDE1F3E0DF011D92DA
:103040008A95E9F7CB2C94C04D875E87DF86702F79
:10305000198B088B6D2D89890E94F015882309F43E
:10306000BBCFDD2009F4B8CF20912203822F8295B7
:103070008F7090E002970CF48ACF80911D0390919D
:103080001E039A8389831B821D830C832E83CE01AA
:1030900001967BCF80959095800F911FA9CFCD2C65
:1030A000DD2009F499CF65132EC034132CC0209174
:1030B000220320FD1FC0822F82958F70D9F0D70187
:1030C00015962C9315978F3049F08F5F982F929516
:1030D000907F822F8F70892B15968C93C7010E9449
:1030E000A41286E0F701ADE1B3E001900D928A955C
:1030F000E1F791CF86E0F701ADE1B3E001900D92E9
:103100008A95E1F735C04D875E87DF86702F198B72
:10311000088B6D2D89890E94F015811138CF80911F
:103120002203816080932203C7010E94A41220C061
:10313000DD2009F451CF4D875E87DF86702F198B14
:10314000088B6D2D89890E94F015882309F444CFDE
:103150001ECF81113DCF0CC0243031050CF03CCF87
:103160009F7009F435CFF7019581907F09F030CF3A
:103170008C2D61960FB6F894DEBF0FBECDBFDF91E8
:10318000CF911F910F91FF90EF90DF90CF90BF9064
:1031900008951F93CF93DF93CDB7DEB72C970FB66B
:1031A000F894DEBF0FBECDBF4F83588769877A87FB
:1031B0008B879C87CE0107960E94F016882369F0C2
:1031C0008F8198852A853B85232BF1F19F3F09F05C
:1031D00063C08F3F09F060C037C086E0FE013796BC
:1031E000DE01119601900D928A95E1F76F81788545
:1031F000EA85FB85309741F17F3F11F46F3F21F164
:103200002091EC0230E0C901019687709927409126
:10321000EB0250E08417950709F447C069837A836D
:10322000FD83EC8396E0929FD001939FB00D112413
:10323000A351BD4FFE01319601900D929A95E1F791
:103240008093EC020E94661616E08091EB0290914A
:10325000EC028917C1F1189FC001112483519D4FC1
:103260000E94F016882379F1E091EB021E9FF00195
:103270001124E351FD4F408151816281738184812A
:1032800095810E9456168091EB0290E0019687701E
:1032900099278093EB02D9CF4F81588569857A852C
:1032A0008B859C850E945616CFCF0E94EC151092FC
:1032B000EC021092EB02EDE1F3E086E0DF011D92FB
:1032C0008A95E9F7C1CF2C960FB6F894DEBF0FBEF2
:1032D000CDBFDF91CF911F910895DF92EF92FF92C2
:1032E0000F931F93CF93DF93FC01892B09F48AC0BE
:1032F000E12CF12CDD24D394EF01219684918537C4
:1033000009F461C058F4843708F04EC0843008F0E6
:103310006AC08130D1F0823071F174C0883709F40D
:103320005DC050F4863709F455C0873709F06AC08C
:103330008E2D0E94591C54C09CE7980F903708F0BE
:1033400061C08F770E946E1250C08F010E5F1F4FB9
:10335000FE01849190E2980F983050F48770FD2D13
:1033600001C0FF0F8A95EAF78F2F0E945F1C14C0DF
:103370000E94C41113C08F010E5F1F4FFE01C49144
:1033800080E28C0F883060F4C7708D2D01C0880FEB
:10339000CA95EAF70E94651C0E94861CE80125C0B8
:1033A0008C2F0E946E12FACF9F012E5F3F4FFE01BD
:1033B000C491CC2369F08FE99FE00197F1F700C039
:1033C0000000C150F6CF9F012E5F3F4FFE01F490E9
:1033D000E9010BC00E94491CE82E07C00E945C1C3A
:1033E0000E94861C02C00E94C4118F2D882341F0C8
:1033F000EFE9FFE03197F1F700C000008150F6CF10
:10340000FE017ACFDF91CF911F910F91FF90EF9046
:10341000DF9008956093A3037093A4038093A503A2
:103420009093A6030C94D81C08956093A7037093FF
:10343000A8038093A9039093AA030C94D71C0F931D
:103440001F930091A7031091A8032091A903309125
:10345000AA03602B712B822B932B6093A70370938D
:10346000A8038093A9039093AA031F910F910C9432
:10347000D71C0F931F930091A7031091A8032091CD
:10348000A9033091AA0360237123822393236093BD
:10349000A7037093A8038093A9039093AA031F9195
:1034A0000F910C94D71C0F931F930091A7031091B9
:1034B000A8032091A9033091AA03602771278227CE
:1034C00093276093A7037093A8038093A903909315
:1034D000AA031F910F910C94D71C60E070E0CB0100
:1034E0000C940A1A0F931F9341E050E060E070E0E3
:1034F0008A019B0104C0000F111F221F331F8A95F0
:10350000D2F7C901B8011F910F910C940A1A0F93B9
:103510001F9341E050E060E070E004C0440F551F8D
:10352000661F771F8A95D2F78091A3039091A40319
:10353000A091A503B091A6038A019B01082B192B2A
:103540002A2B3B2BC901B8011F910F910C940A1A29
:103550000F931F9341E050E060E070E004C0440F1F
:10356000551F661F771F8A95D2F740955095609535
:1035700070958091A3039091A403A091A503B091AD
:10358000A6038A019B01082319232A233B23C9018F
:10359000B8011F910F910C940A1A0F931F9341E0E9
:1035A00050E060E070E004C0440F551F661F771FB5
:1035B0008A95D2F78091A3039091A403A091A503CB
:1035C000B091A6038A019B01082719272A273B27C8
:1035D000C901B8011F910F910C940A1A0F931F9300
:1035E0000091A3031091A4032091A5033091A60399
:1035F000602B712B822B932B1F910F910C940A1A25
:103600000F931F930091A3031091A4032091A5038E
:103610003091A60360237123822393231F910F917E
:103620000C940A1A0F931F930091A3031091A40303
:103630002091A5033091A603602771278227932745
:103640001F910F910C940A1A08958F929F92AF9236
:10365000BF92DF92EF92FF920F931F93CF93DF936E
:1036600000D000D01F92CDB7DEB76B837C838D83F3
:103670008A018C819D81892B21F01F3F29F44F3FC6
:1036800019F480E090E04CC08B818823C9F18090D0
:10369000A7039090A803A090A903B090AA038091DB
:1036A000A3039091A403A091A503B091A603882A37
:1036B000992AAA2ABB2A8FE1E82EF12CD501C40150
:1036C0000E2C04C0B695A795979587950A94D2F7C6
:1036D00080FF07C0DE2CB8018E2D0E94F61D0197D9
:1036E00029F481E0E81AF10848F7D12C88E0189F06
:1036F000F0011124E00FF11DED5DFC4FD08209C0F7
:1037000088E0189FF0011124E00FF11DED5DFC4FE2
:10371000D08009831A8369817A818D2D0E94F61DDC
:103720000F900F900F900F900F90DF91CF911F91FE
:103730000F91FF90EF90DF90BF90AF909F908F9090
:10374000089590911401992321F090911501911100
:1037500009C02091160130911701F90132969FEFAF
:1037600040E030C0982F9695969596959F31A0F49D
:10377000E0911601F0911701E90FF11D877021E02A
:1037800030E0A90102C0440F551F8A95E2F7CA0133
:103790009181892B818308959091CE0390FF23C05E
:1037A0001F928F9389E094E09F938F930E94190654
:1037B0000F900F900F900F9008959F3F39F04F5F3B
:1037C0004E3141F051915813F8CF0DC05111F7CF40
:1037D000942FF5CF9F3F39F0F901E90FF11D97FDC7
:1037E000FA9582830895089590911401992321F008
:1037F00090911501911109C0209116013091170186
:10380000F9013296205E3F4F30C0982F96959695DD
:1038100096959F31A8F4E0911601F0911701E90FF8
:10382000F11D877021E030E0A90102C0440F551F4F
:103830008A95E2F7CA018095918189238183089551
:103840009091CE0390FF16C01F928F938BEE93E062
:103850009F938F930E9419060F900F900F900F90D7
:1038600008953196E217F30729F090819813F9CF64
:103870001082F7CF089581E090E0E0911601F09179
:103880001701E80FF91F1082019680329105A9F700
:1038900008958091CD0308959091CD03892B809355
:1038A000CD03089580959091CD0389238093CD0316
:1038B00008958093CD0308951092CD0308959091BB
:1038C000CC03892B8093CC03089580959091CC03F1
:1038D00089238093CC0308951092CC03089580939C
:1038E000AB0308951092AB03089580911601909157
:1038F0001701FC0131969C01205E3F4F80E09191C1
:1039000091118F5FE217F307D1F70895E091160147
:10391000F09117018091CD038083E0911601F09121
:10392000170190818091CC03892B80838091AB0318
:10393000882361F0E0911601F09117019081892BA5
:1039400080830E94751C81111092AB038091160137
:10395000909117010C94D70F90938B0180938A015B
:1039600008958295982F9C7C392F36953695282F6F
:10397000237344E0249FC0011124932F982B292FF7
:103980002A7A2695892F8575880F822B08950895A8
:10399000CF93DF9300D000D01F92CDB7DEB70F904A
:1039A0000F900F900F900F90DF91CF910895089591
:1039B00008950C9430118091E303843021F110922A
:1039C000CF0320E488E190E00FB6F894A8958093A7
:1039D00060000FBE2093600083B7817F846083BF47
:1039E00083B7816083BF7894889583B78E7F83BFC8
:1039F0000FB6F894A895809160008861809360006C
:103A0000109260000FBE0895CF930E9482110E9411
:103A100024070E948311C0E08C2F0E94A607811109
:103A200004C0CF5FC031C1F701C081E0CF910895DC
:103A30000E94AC070C94EC151F920F920FB60F92D8
:103A400011248F939F93AF93BF938091CF038111E4
:103A500013C08091D0039091D103A091D203B09173
:103A6000D3034196A11DB11D8093D0039093D10340
:103A7000A093D203B093D303BF91AF919F918F9145
:103A80000F900FBE0F901F90189582E084BD93E0B9
:103A900095BD9AEF97BD80936E0008952FB7F89467
:103AA0008091D0039091D103A091D203B091D30320
:103AB0002FBF08952FB7F8946091D0037091D10370
:103AC0008091D2039091D3032FBF0895CF92DF92BC
:103AD000EF92FF920F931F932FB7F8944091D0036A
:103AE0005091D1036091D2037091D3032FBF6A012B
:103AF0007B01EE24FF248C0120E030E0C016D106CB
:103B0000E206F30610F4415051099A01281B390BC3
:103B1000C9011F910F91FF90EF90DF90CF90089512
:103B20001F920F920FB60F9211248F939F93AF9312
:103B3000BF938091D0039091D103A091D203B09113
:103B4000D3030196A11DB11D8093D0039093D1039F
:103B5000A093D203B093D303BF91AF919F918F9164
:103B60000F900FBE0F901F9018950E94E40CF894D0
:103B70002FEF87EA91E6215080409040E1F700C0A6
:103B8000000087E090EBDC018093EC039093ED0361
:103B9000A093EE03B093EF039CE088E10FB6F89496
:103BA000A895809360000FBE90936000FFCF80E0E7
:103BB00090E008950895E72FF0E090E1899FE00DEF
:103BC000F11D112483E0EE0FFF1F8A95E1F7E60F48
:103BD000F11DE052FF4F84910895E82FF0E0EE0FC1
:103BE000FF1FE05AF0408591949108950E94DB1DDB
:103BF00090E4980F903218F40E94ED1D08958D3BCB
:103C000050F4883AA0F5853A28F5843000F58130E3
:103C100009F49DC099C0883E98F4803EC0F48F3B63
:103C200009F092C00E94EC152FEF80E792E021503E
:103C300080409040E1F700C000000E94B51D84C0A4
:103C4000803F08F481C0282F30E0306582C0282FE3
:103C500030E07FC0853A29F0863A31F023E830E43D
:103C600078C021E830E475C022E830E472C0883AB8
:103C700061F1893A69F18A3A71F18B3A79F18C3ABA
:103C800081F18D3A89F18E3A91F18F3A99F1813B28
:103C9000A1F1803BA9F1823BB1F1833BB9F1843BB7
:103CA000C1F1853BC9F1863BD1F1873BD9F1883B16
:103CB000E1F1893BE9F18A3BF1F18B3BF9F18C3B76
:103CC00009F43FC020E034E444C022EE34E441C0B3
:103CD00029EE34E43EC02AEE34E43BC025EB34E464
:103CE00038C026EB34E435C023EB34E432C024EB97
:103CF00034E42FC027EB34E42CC02CEC34E429C08E
:103D00002DEC34E426C023E835E423C02AE835E46A
:103D100020C022E935E41DC024E935E41AC021E2BF
:103D200036E417C023E236E414C024E236E411C0BE
:103D300025E236E40EC026E236E40BC027E236E484
:103D400008C02AE236E405C020E030E002C021E0ED
:103D500030E0C90108958091D60380FF0BC06091C7
:103D60001B0185E0689FB0011124759567957595D5
:103D700067952BC081FF09C060911B0185E0689F9A
:103D8000B00111247595679520C082FF07C060912E
:103D90001B0185E0689FB001112417C09091D703E3
:103DA0009923D1F060911A01961788F720911B0191
:103DB00085E0289F90011124929FA001939F500DB0
:103DC000112470E0CA010E9479266038710540F420
:103DD0006115710539F002C065E070E0862F089525
:103DE0008FE7089581E008958091D60380FF08C091
:103DF0006091190170E0759567957595679521C07B
:103E000081FF06C06091190170E07595679519C032
:103E100082FF04C06091190170E010C09091D70337
:103E20009923C1F0609118019617A0F780911901AC
:103E3000899FC001112470E00E94792660387105C5
:103E400028F46115710521F0862F08958FE70895F4
:103E500081E0089561E070E0F4CF803F21F40E949A
:103E6000AB1E819504C0813F29F40E94AB1E809354
:103E7000DA030895823F21F40E94AB1E819504C0AD
:103E8000833F29F40E94AB1E8093D9030895893F94
:103E900019F40E94F41E05C08A3F31F40E94F41EFA
:103EA00081958093DB0308958B3F21F40E94F41EDB
:103EB000819504C08C3F29F40E94F41E8093DC039A
:103EC0000895843F21F48091D803816017C0853F15
:103ED00021F48091D803826011C0863F21F4809143
:103EE000D80384600BC0873F21F48091D803886099
:103EF00005C0883F31F48091D80380618093D80356
:103F000008958D3F21F48091D60381600BC08E3FD0
:103F100021F48091D603826005C08F3F29F48091FF
:103F2000D60384608093D6030895803F39F480914E
:103F3000DA0387FF6CC01092DA0369C0813F29F46D
:103F40008091DA031816BCF362C09091D903823FC6
:103F500029F497FF5CC01092D90359C0833F19F42C
:103F60001916CCF354C0893F41F48091DB03181635
:103F70000CF04DC01092DB034AC08A3F29F48091B7
:103F8000DB0387FF44C0F6CF8B3F39F48091DC031D
:103F900087FF3DC01092DC033AC08C3F29F480912A
:103FA000DC031816BCF333C0843F21F48091D8039E
:103FB0008E7F17C0853F21F48091D8038D7F11C07B
:103FC000863F21F48091D8038B7F0BC0873F21F47B
:103FD0008091D803877F05C0883F31F48091D80352
:103FE0008F7E8093D80313C08D3F21F48091D60338
:103FF0008E7F0BC08E3F21F48091D6038D7F05C04C
:104000008F3F29F48091D6038B7F8093D6038091D4
:10401000D90381110EC08091DA0381110AC0809109
:10402000DB03811106C08091DC03811102C0109274
:10403000D70308958091CE0383FF7EC08EE494E081
:104040000E9480058091D8031F928F9389E494E0A9
:104050009F938F930E94190687E494E00E94800545
:104060008091D903282F082E000C330B3F938F9398
:1040700084E494E09F938F930E94190682E494E075
:104080000E9480058091DA03282F082E000C330B44
:104090003F938F938FE394E09F938F930E94190631
:1040A0008DE394E00E9480058091DB03282F082E89
:1040B000000C330B3F938F938AE394E09F938F938D
:1040C0000E94190688E394E00E9480058091DC0339
:1040D000282F082E000C330B3F938F9385E394E039
:1040E0009F938F930E94190682E394E00E948005BB
:1040F0008091D7031F928F938FE294E09F938F93C9
:104100000E9419068DE294E00E9480058091D603FA
:104110001F928F938AE294E09F938F930E941906D7
:1041200087E294E00E9480058DB79EB74C960FB64B
:10413000F8949EBF0FBE8DBF88ED93E00E942010C3
:104140000E944E1D9093D5038093D40308951F932E
:10415000CF93DF938091D4039091D5030E94661D85
:10416000AC019091D703992321F020911C0130E0FC
:1041700006C020911D018AE0289F9001112442175A
:10418000530708F485C08091D903C091DA03D09118
:10419000DB031091DC03811107C0C11175C0D1117F
:1041A00073C0111171C074C09F3F19F09F5F90934D
:1041B000D703181624F40E94AB1E8093D903809174
:1041C000D90387FF05C00E94AB1E81958093D90358
:1041D0001C1624F40E94AB1E8093DA038091DA034C
:1041E00087FF05C00E94AB1E81958093DA03609122
:1041F000D903662331F1C091DA03CC2311F1062EE5
:10420000000C770B880B990B0E94802523E333E386
:1042100043E35FE30E94E4250E9448256093D903AD
:104220006C2FCC0F770B880B990B0E94802523E312
:1042300033E343E35FE30E94E4250E944825609353
:10424000DA031D1624F40E94F41E8093DB03809190
:10425000DB0387FF05C00E94F41E81958093DB037A
:10426000111624F40E94F41E8093DC038091DC0379
:1042700087FF05C00E94F41E81958093DC03DF91C7
:10428000CF911F910C941A209F3F09F08FCF97CFA9
:10429000DF91CF911F910895E8EDF3E085E0DF0114
:1042A0001D928A95E9F71092D7031092D6030895CC
:1042B00081E796E00E9480051F9281E08F931F9214
:1042C00085E08F9383E296E09F938F930E94190677
:1042D0000F900F900F900F900F900F9008958330D4
:1042E000E9F128F4813061F0823009F108958530D8
:1042F00009F462C008F449C0863009F474C0089516
:1043000080911D01262F30E0280F311D2F3F3105F0
:1043100024F4680F60931D0103C08FEF80931D018B
:1043200080911D011F928F938CE595E072C0809162
:104330001C01262F30E0280F311D2F3F310524F4BA
:10434000680F60931C0103C08FEF80931C01809164
:104350001C011F928F938AE495E05BC080911B0142
:10436000262F30E0280F311D2F3F310524F4680F30
:1043700060931B0103C08FEF80931B0180911B0191
:104380001F928F9387E395E044C080911A01262FF6
:1043900030E0280F311D2F3F310524F4680F609362
:1043A0001A0103C08FEF80931A0180911A011F92A6
:1043B0008F9382E295E02DC080911901262F30E085
:1043C000280F311D2F3F310524F4680F6093190128
:1043D00003C08FEF80931901809119011F928F9371
:1043E00089E095E016C080911801262F30E0280F53
:1043F000311D2F3F310524F4680F6093180103C06D
:104400008FEF80931801809118011F928F938EEE89
:1044100094E09F938F930E9419060F900F900F9036
:104420000F900895833081F128F4813059F0823063
:10443000D1F00895853009F449C0B8F1863009F407
:1044400056C0089580911D01681720F4861B809343
:104450001D0102C010921D0180911D011F928F93BA
:104460008FED94E054C080911C01681720F4861BE6
:1044700080931C0102C010921C0180911C011F92AC
:104480008F938DEC94E043C080911B01681720F45A
:10449000861B80931B0102C010921B0180911B019F
:1044A0001F928F938AEB94E032C080911A016817B3
:1044B00020F4861B80931A0102C010921A01809189
:1044C0001A011F928F9385EA94E021C0809119010F
:1044D000681720F4861B8093190102C010921901FD
:1044E000809119011F928F938CE894E010C0809105
:1044F0001801681720F4861B8093180102C01092DF
:104500001801809118011F928F9381E794E09F9387
:104510008F930E9419060F900F900F900F9008959F
:10452000CF93C82F1F928F9386E797E09F938F9327
:104530000E94190681E090E0A0E0B0E0BC01CD014E
:1045400004C0660F771F881F991FCA95D2F70E9473
:10455000151A0F900F900F900F90CF910C94EC15AF
:10456000CF938732A8F58E3108F02BC1803109F442
:104570009FC0F8F4873009F464C0A8F4863009F0CD
:1045800024C18091CE03817F8E7F8093CE038BE701
:1045900097E00E94800582E59AE00E94800581E014
:1045A0008093DE034CC08B30F1F18E3009F46CC087
:1045B0000CC1863109F4B0C020F4813109F4EDC09A
:1045C00004C1893109F491C08B3109F449C0FDC09F
:1045D000883349F150F4893209F4F1C0853309F484
:1045E000EEC0873209F0F1C0EAC0833409F4E7C0B5
:1045F00028F48A3308F4E9C08953E4C0883409F008
:10460000E4C00E94EC1581E49AE00E9480052FEF3F
:1046100083ED90E3215080409040E1F700C000001E
:104620000E94B51D0CC082EA97E05CC088E29AE067
:104630000E9480058091CE0381608093CE03C1E00B
:10464000C9C08091CE03C82FC17080FFEFCF84E333
:104650009AE00E9480058091CE03817F8E7F3DC0CD
:104660009091CE0391FBCC27C0F981E0C827892F18
:10467000C0FB81F98093CE03CC2319F08BE19AE043
:1046800027C08DE09AE02EC09091CE0392FBCC27FC
:10469000C0F981E0C827892FC0FB82F98093CE033F
:1046A000CC2319F08EEF99E013C08EEE99E01AC07A
:1046B0009091CE0393FBCC27C0F981E0C827892FC6
:1046C000C0FB83F98093CE03CC2351F082EE99E0B6
:1046D0000E9480058091CE0381608093CE037AC0D2
:1046E00085ED99E00E948005AACF86EC99E00E94B2
:1046F000800584EA99E00E94800580E699E00E94A6
:10470000800589E399E00E9480058EEF98E00E9481
:10471000800580ED98E0E6CF82EC98E00E9480056D
:104720000E94CB0F1F928F9388EA98E09F938F93FC
:104730000E941906809114011F928F9381E998E0DD
:104740009F938F930E9419068091D3021F928F939B
:104750008EE798E09F938F930E9419068091150130
:104760001F928F938BE698E09F938F930E94190678
:104770000E945A1D9F938F937F936F9384E598E0D7
:104780009F938F930E9419068DB79EB746960FB6DA
:10479000F8949EBF0FBE8DBF52CF0E94EC15C09102
:1047A000150181E0C827C0931501CC2329F08AE4C4
:1047B00098E00E9480050EC08FE398E093CF80E0E0
:1047C00001C08D510E9490223ACF8DE398E00E9463
:1047D0008005C0E08C2FCF91089580E0089580E09F
:1047E0000895CF93C82F8091DE03813079F020F0B7
:1047F000823009F44DC044C1E0911601F0911701D7
:1048000080818152823008F03DC108C0E0911601DC
:10481000F091170180818152823060F48C2F0E94C8
:10482000ED23811104C08C2F0E94B0222FC081E0A3
:1048300090E02CC08C2F0E94EF23811126C0C43140
:10484000E1F070F4CB3081F0C031D1F40E945821F6
:104850008EE697E00E94800582E08093DE0315C01B
:10486000C93259F0C83361F48BE797E00E948005A4
:1048700082E797E00E94800508C01092DE0304C121
:104880008CE697E00E948005FFC081E08170FEC049
:10489000C43228F5CE3108F0C1C0CB30A1F1D0F43C
:1048A000C73009F0D3C08EE180931D0182E380936D
:1048B0001C018AE080931B0184E180931A0188E047
:1048C0008093190188E28093180182E196E00E94AA
:1048D0008005BFC0C33149F1C431C1F0B7C0CB348A
:1048E00009F4A9C028F4C93289F0C83361F0AEC018
:1048F000C13509F49EC0C23509F499C0CE3409F01F
:10490000A5C06AE09EC00E945821A3C08091DD032B
:10491000882319F01092DD039CC08FE196E00E947D
:10492000800581E08093DE03B1C089EF95E00E94AD
:10493000800587EE95E00E94800580911D011F9201
:104940008F9384EE95E09F938F930E94190682EED9
:1049500095E00E94800580ED95E00E9480058091A1
:104960001C011F928F938DEC95E09F938F930E9473
:1049700019068BEC95E00E9480058CEB95E00E9477
:10498000800580911B011F928F9389EB95E09F9387
:104990008F930E94190687EB95E00E94800586EAB6
:1049A00095E00E94800580911A011F928F9383EAFF
:1049B00095E09F938F930E94190681EA95E00E94EB
:1049C00080058CE895E00E948005809119011F9276
:1049D0008F9389E895E09F938F930E94190687E84B
:1049E00095E00E94800580E795E00E948005809117
:1049F00018011F928F938DE695E09F938F930E94ED
:104A000019068BE695E00E9480058DB79EB7489603
:104A10000FB6F8949EBF0FBE8DBF1BC0CE51EC2FBA
:104A2000F0E0E058FE4F80818093DD0312C061E02A
:104A300003C061E006C06AE08091DD030E946F213F
:104A400008C08091DD030E94122203C080E196E03D
:104A500013C08091DD03882369F01F928F938AE051
:104A600096E09F938F930E9419060F900F900F90DE
:104A70000F9004C087E096E00E94800581E006C0A8
:104A80001092DE0380E002C080E000CFCF91089555
:104A90000E944F256894B1110C94DE2508950E9460
:104AA000C32588F09F5798F0B92F9927B751B0F0D8
:104AB000E1F0660F771F881F991F1AF0BA95C9F7A2
:104AC00014C0B13091F00E94DD25B1E008950C943E
:104AD000DD25672F782F8827B85F39F0B93FCCF3F1
:104AE000869577956795B395D9F73EF4909580951F
:104AF000709561957F4F8F4F9F4F0895E89409C03F
:104B000097FB3EF490958095709561957F4F8F4F00
:104B10009F4F9923A9F0F92F96E9BB279395F69516
:104B2000879577956795B795F111F8CFFAF4BB0F94
:104B300011F460FF1BC06F5F7F4F8F4F9F4F16C0F8
:104B4000882311F096E911C0772321F09EE8872F82
:104B5000762F05C0662371F096E8862F70E060E03E
:104B60002AF09A95660F771F881FDAF7880F9695B7
:104B7000879597F9089557FD9058440F551F59F0A0
:104B80005F3F71F04795880F97FB991F61F09F3F3A
:104B900079F087950895121613061406551FF2CF63
:104BA0004695F1DF08C0161617061806991FF1CFB3
:104BB00086957105610508940895E894BB276627DA
:104BC0007727CB0197F908950E94F7250C94682662
:104BD0000E945A2638F00E94612620F0952311F099
:104BE0000C9451260C94572611240C94DE250E9417
:104BF000BB2570F3959FC1F3950F50E0551F629F41
:104C0000F001729FBB27F00DB11D639FAA27F00D25
:104C1000B11DAA1F649F6627B00DA11D661F829F4C
:104C20002227B00DA11D621F739FB00DA11D621F31
:104C3000839FA00D611D221F749F3327A00D611D4E
:104C4000231F849F600D211D822F762F6A2F112430
:104C50009F5750409AF0F1F088234AF0EE0FFF1F63
:104C6000BB1F661F771F881F91505040A9F79E3FBA
:104C7000510580F00C9451260C94DE255F3FE4F33F
:104C8000983ED4F3869577956795B795F795E79510
:104C90009F5FC1F7FE2B880F911D9695879597F919
:104CA000089597F99F6780E870E060E008959FEFAE
:104CB00080EC089500240A941616170618060906B3
:104CC000089500240A941216130614060506089582
:104CD000092E0394000C11F4882352F0BB0F40F40A
:104CE000BF2B11F460FF04C06F5F7F4F8F4F9F4F4A
:104CF000089597FB072E16F4009407D077FD09D08E
:104D00000E94932607FC05D03EF4909581959F4F15
:104D10000895709561957F4F0895EE0FFF1F0590E0
:104D2000F491E02D0994AA1BBB1B51E107C0AA1FF7
:104D3000BB1FA617B70710F0A61BB70B881F991F3C
:104D40005A95A9F780959095BC01CD010895F894E6
:024D5000FFCF93
:104D52008E0100000FB2010000FFB50743082008D2
:104D6200EC07B8070101AC032808140A321E6F7A57
:104D72000000000000000000000000000000000031
:104D8200000000000000007F00547C0000000000D2
:104D920000000000000000005574607700610063AD
:104DA200007562787172000000000000005A5B5CBE
:104DB2005D5E0000005F404D36223953030603D08A
:104DC20002AE027502E80101021A02330253020026
:0A4DD20001020304050607080900AA
:00000001FF
